:020000000829CD
:1000080008002C08A0002D08A1000130A2006400FF
:100018003120031C1E28A20B0B28FF30A007031C4D
:10002800A107031C0329FA30A2000B286400312021
:1000380003181A288320A8010830A300842031203F
:100048000318A80AAB1EA801A20CA30B2228AB1AFE
:10005800A21384200314220808003A0884003808F0
:1000680084178004841300052B1B3806FF3E080004
:10007800A4002908031403190329FE20031C0800FF
:10008800A000251883172408840020088000831303
:10009800A40AA9033D280408A6003A088400F03001
:1000A800B7050830A70003100318B70A6920A60C83
:1000B800A70B58280000AB1A370C69200621031437
:1000C80069202F08A3002E08AA288413AB1F7828BC
:1000D800000838042B1F38068000841700083804ED
:1000E800031C38068000842800083804031C3806DE
:1000F8002B1B380680008417380980058428371799
:100108002B081F39003EA1002A080E3E0318A10A39
:10011800371FB7283713A0000230C920B728A4001A
:1001280029080319032925188317240884000008BF
:100138008313FE20A40AA903942803178D008316AD
:100148008C130C1483120C080329A301A200FF309E
:10015800A207031CA307031C03290330A100E730EF
:10016800B720AB28A101FC3EA000A109031CC228AE
:10017800FF300000A0070318BD28A0076400A10FE6
:10018800BC2808000310A10CA00CFF3E0318C628C9
:1001980020080329A101A301A2000130D828A10148
:1001A800A301A2000430D828A80023082102031DB7
:1001B800DF28220820020430031801300319023016
:1001C8002805031DFF3003291030A800A101A00154
:1001D800A70CA60C031CF6282208A007230803185E
:1001E800230FA107A10CA00CA50CA40CA80BEC28AC
:1001F80024080329840031088A0030088200831308
:100208000313831264000800831607309F008616C4
:100218000617861706108610061186110612880121
:100228000710871007118711071287128312C80158
:10023800BE018801C301C501C601C101C70188010A
:1002480087100711071086140611C901C001871607
:1002580064308A01A92087120A308A01A9208716EA
:100268000230A30058308A01AA208A110A12902E5F
:10027800071406308A01B620071008008710861474
:1002880006110130C3006400033043028A110A12C8
:10029800031870293E308800C03088008A013C214C
:1002A800403088008A013C21B83088008A013C210E
:1002B8003F3088008A013C21831086188314061970
:1002C8008614061D861083180615831C0611C30A9A
:1002D8008A110A12031D472986140611080087107F
:1002E8003E3088008A013C21861406110130C30083
:1002F8006400033043028A110A120318BE29B83079
:10030800C5006400C03045028A110A120318AE29DC
:1003180087108A013C21403088008A013C21450829
:1003280088008A013C2187140130C60064004130EE
:1003380046028A110A120318A92988018A013C2158
:10034800C60A8A110A12031D9A29C50A8A110A12B5
:10035800031D852983108618831406198614061D23
:10036800861083180615831C0611C30A8A110A12FF
:10037800031D7C29861006158710B83088008A016D
:100388003C21C03088008A013C21403088008A0125
:100398003C2186140611B83088008A013C21C030FF
:1003A80088008A013C21403088008A013C213F3086
:1003B80088008A013C2187148614061108008714D6
:1003C800D8303E07B200FF300318013EB3003208B0
:1003D800A6003308A7000530A200A3018A01E8207F
:1003E800BE0004303E07C6003E08C500640045084C
:1003F80046028A110A12031C102A8A110A121C22A8
:1004080045088A01A12088008A013C21C10AC50A41
:100418008A110A12031DFA298A110A1214220800E5
:100428008A110A121C2288018A013C21C10A08008B
:1004380064004108403C8A110A12031D2B2A8610C9
:1004480006158710403088008A013C218714640013
:100458004108803C8A110A12031D3C2A86140611A1
:10046800C70AC1018710403088008A013C218714DF
:1004780064004708083C8A110A12031D4D2AC70167
:1004880064004A08013C8A110A12031D4D2A0730EC
:10049800C7008710B830470788008A013C218714B5
:1004A800080064003F3041028A110A120318632AC7
:1004B800861406114108C0008A110A12682A86109B
:1004C800061540304102C0008710B8304707880041
:1004D8008A013C214030400788008A013C2187146A
:1004E80008000830C100C7018A015522C301640011
:1004F800143043028A110A120318C82A4308133C0D
:100508008A110A12031CA72A8A110A128F22BE0016
:100518008A110A12A72A02308A0043088207473440
:1005280052344134503448344934433420344C3400
:100538004334443420345434453452344D344934EB
:100548004E3441344C3464003E08203C8A110A126F
:10055800031DC12A0130C5006400043045028A1118
:100568000A120318BE2A8A011422C50A8A110A121D
:10057800031DB02A8A110A12C32A8A01E321C30A79
:100588008A110A12031D7B2A0130C5006400053058
:1005980045028A110A120318022BC1014508C70037
:1005A8008A015522C3016400403043028A110A12AD
:1005B8000318E72A143088008A013C21C30A8A11EB
:1005C8000A12031DD72A4030C1008A015522C301EF
:1005D8006400803043028A110A120318FC2A14307E
:1005E80088008A013C21C30A8A110A12031DEC2AD9
:1005F8000330C5078A110A12031CCA2AC101053033
:10060800C7008A015522C3016400163043028A11CB
:100618000A120318572B4308153C8A110A12031CA7
:10062800362B8A110A121C23BE008A110A12362B95
:1006380003308A0043088207533445344E34443427
:10064800203443344D3444345334203456344934FC
:10065800413420345434453452344D3449344E34C2
:1006680041344C3464003E08203C8A110A12031DB0
:10067800502B0130C5006400043045028A110A126B
:1006880003184D2B8A011422C50A8A110A12031D68
:100698003F2B8A110A12522B8A01E321C30A8A11BD
:1006A8000A12031D082BC1010630C7008A01552212
:1006B800C3016400403043028A110A1203186D2BEB
:1006C8003C3088008A013C21C30A8A110A12031DA2
:1006D8005D2B4030C1008A015522C301640080307F
:1006E80043028A110A120318822B3C3088008A01BF
:1006F8003C21C30A8A110A12031D722BC101023060
:10070800C7008A015522C30164000A3043028A11D6
:100718000A120318CB2B4308093C8A110A12031C3E
:10072800AA2B8A110A129C23BE008A110A12AA2B2C
:1007380003308A004308820750344F34523454340B
:1007480042342034503449344E34533464003E0823
:10075800203C8A110A12031DC42B0130C500640015
:10076800043045028A110A120318C12B8A01142287
:10077800C50A8A110A12031DB32B8A110A12C62B45
:100788008A01E321C30A8A110A12031D882B40300B
:10079800C1000230C7008A015522C30164000B3032
:1007A80043028A110A120318162C43080A3C8A11BC
:1007B8000A12031CF52B8A110A12E623BE008A11BD
:1007C8000A12F52B03308A004308820750344F344D
:1007D800523454344334203453345434413454342C
:1007E800453464003E08203C8A110A12031D0F2C70
:1007F8000130C5006400043045028A110A1203184A
:100808000C2C8A011422C50A8A110A12031DFE2B18
:100818008A110A12112C8A01E321C30A8A110A12C9
:10082800031DD22B0800861006150130C300640092
:10083800033043028A110A1203184C2C8710BF3068
:1008480088008A013C21403088008A013C218714B5
:10085800C5016400413045028A110A1203183C2C74
:1008680088018A013C21C50A8A110A12031D2D2C10
:1008780083108618831406198614061D861083189B
:100888000615831C0611C30A8A110A12031D1B2CA4
:1008980086140611C1010730C700080064003C082F
:1008A800423C8A110A12031D702D30303D02C200ED
:1008B80064004208003C8A110A12031D852C01308D
:1008C80086068316061083124708CB004108CC0021
:1008D8000330C700C1018A01552264008A110A1237
:1008E800061C7B2C3130BE008A110A127D2C303058
:1008F800BE008A01E3214B08C7004C08C1008A01E9
:10090800552264004208033C8A110A12031DB42CC4
:1009180008308606831686110130831286068316F0
:10092800061083124708CB004108CC000330C700EB
:100938000830C1008A01552264008A110A12861DF6
:10094800AA2C3130BE008A110A12AC2C3030BE00FD
:100958008A01E3214B08C7004C08C1008A015522CF
:1009680064004208043C8A110A12031DE32C10306B
:100978008606831606120130831286068316061031
:1009880083124708CB004108CC000330C70012305F
:10099800C1008A01552264008A110A12061ED92C48
:1009A8003130BE008A110A12DB2C3030BE008A01B9
:1009B800E3214B08C7004C08C1008A015522640096
:1009C8004208053C8A110A12031D122D20308606A2
:1009D8008316861201308312860683160610831248
:1009E8004708CB004108CC000330C7001C30C100C9
:1009F8008A01552264008A110A12861E082D313098
:100A0800BE008A110A120A2D3030BE008A01E32185
:100A18004B08C7004C08C1008A01552264004208EF
:100A2800063C8A110A12031D412D403086068316A2
:100A380006130130831286068316061083124708B0
:100A4800CB004108CC000330C7002630C1008A0122
:100A5800552264008A110A12061F372D3130BE0054
:100A68008A110A12392D3030BE008A01E3214B0861
:100A7800C7004C08C1008A01552264004208073C9F
:100A88008A110A12031D702D80308606831686137C
:100A98000130831286068316061083124708CB009E
:100AA8004108CC000330C7003030C1008A0155220C
:100AB80064008A110A12861F662D3130BE008A1121
:100AC8000A12682D3030BE008A01E3214B08C700A6
:100AD8004C08C1008A0155224230BE000800470870
:100AE800CB004108CC003E08CD000330C700C1014F
:100AF8008A01552264008A110A12061C882D313099
:100B0800BE008A110A128A2D3030BE008A01E32104
:100B18000830C1008A01552264008A110A12861D14
:100B28009A2D3130BE008A110A129C2D3030BE0039
:100B38008A01E3211230C1008A01552264008A111A
:100B48000A12061EAC2D3130BE008A110A12AE2DD3
:100B58003030BE008A01E3211C30C1008A015522D1
:100B680064008A110A12861EBE2D3130BE008A1119
:100B78000A12C02D3030BE008A01E3212630C100A0
:100B88008A01552264008A110A12061FD02D3130BD
:100B9800BE008A110A12D22D3030BE008A01E3212C
:100BA8003030C1008A01552264008A110A12861F5A
:100BB800E22D3130BE008A110A12E42D3030BE0019
:100BC8008A01E3214B08C7004C08C1004D08BE004C
:100BD8008A01552208004708CB004108CC003E088E
:100BE800CD000330C7004030C1008A01552264009F
:100BF8008A110A12071C052E3130BE008A110A120A
:100C0800072E3030BE008A01E3214830C1008A0136
:100C1800552264008A110A12871C172E3130BE0033
:100C28008A110A12192E3030BE008A01E321503091
:100C3800C1008A01552264008A110A12071D292E53
:100C48003130BE008A110A122B2E3030BE008A01C4
:100C5800E3215830C1008A01552264008A110A1222
:100C6800871D3B2E3130BE008A110A123D2E3030CE
:100C7800BE008A01E3216030C1008A015522640068
:100C88008A110A12071E4D2E3130BE008A110A122F
:100C98004F2E3030BE008A01E3216830C1008A013E
:100CA800552264008A110A12871E5F2E3130BE0059
:100CB8008A110A12612E3030BE008A01E321703099
:100CC800C1008A01552264008A110A12071F712E79
:100CD8003130BE008A110A12732E3030BE008A01EC
:100CE800E3217830C1008A01552264008A110A1272
:100CF800871F832E3130BE008A110A12852E3030AC
:100D0800BE008A01E3214B08C7004C08C1004D080A
:100D1800BE008A01552208008A0142218A017321F6
:100D28008A0175228A017325C1010730C7008A012B
:100D38005522861406118710403088008A013C210C
:100D4800BF3088008A013C2187140130CA0007306F
:100D5800BA004030B8005430AA00AB01AE01AF0170
:100D680052308A01502045308A01502041308A0192
:100D7800502044308A01502059308A0150203A309E
:100D88008A0150200A308A0150200D308A015020F3
:100D98008A0173258A01EF250730BA008030B80030
:100DA8005430AA00AB01F430AC000130AD008A0128
:100DB80005208A110A12031CCC2EBE0064003E08CE
:100DC8005D3C8A110A12031D3B2F0730BA004030E0
:100DD800B8005430AA00AB01AE01AF0143308A011C
:100DE80050204D308A01502044308A0150203A303A
:100DF8008A0150200730BA008030B8005430AA0069
:100E0800AB018A011A20403C8A110A12031D052FE2
:100E18000230A9001A30B000B101A5013C308A01A6
:100E28003C200730BA004030B8005430AA00AB016B
:100E3800AE01AF0143308A0150204D308A01502065
:100E480044308A0150203A308A0150200230A900EB
:100E58004F30B000B101A5013C308A0193200A301F
:100E68008A0150200D308A0150208A0152246400E2
:100E78003E08203C8A110A12031D442F8A011422BD
:100E88003E08A00028308A01D320B2003E08A00006
:100E98005A308A01CE20B400320834048A110A126A
:100EA800031DCC2E8A01E3210630C9076400803077
:100EB80049028A110A12031C642F8A011724C901E6
:0A0EC8008A01CC2E63008A01662F18
:02400E00753DFE
:00000001FF
